:020000021000EC
:10E000000C9446F00C9465F00C9465F00C9465F05B
:10E010000C9465F00C9465F00C9465F00C9465F02C
:10E020000C9465F00C9465F00C9465F00C9465F01C
:10E030000C9465F00C9465F00C9465F00C9465F00C
:10E040000C9465F00C9465F00C9465F00C9465F0FC
:10E050000C9465F00C9465F00C9465F00C9465F0EC
:10E060000C9465F00C9465F00C9465F00C9465F0DC
:10E070000C9465F00C9465F00C9465F00C9465F0CC
:10E080000C9465F00C9465F00C9465F011241FBE9F
:10E09000CFEFD0E1DEBFCDBF11E0A0E0B1E0E6E61A
:10E0A000F4EE01E00BBF02C007900D92A030B10763
:10E0B000D9F711E0A0E0B1E001C01D92A230B10794
:10E0C000E1F70E9468F10C9431F20C9400F0BC016D
:10E0D00085E08EBD86B7846086BF80919B0087FDFA
:10E0E00003C006B602FEF9CF06B602FC36C0309178
:10E0F0009C0086B7846086BF1DBC1CBC80919B00C1
:10E1000087FD03C006B602FEF9CF06B602FC25C0A5
:10E1100020919C00932F80E0AC01420F511D20E024
:10E1200030E017C086B7846086BF1DBC1CBC8091E0
:10E130009B0087FD03C006B602FEF9CF06B602FCBF
:10E140000CC080919C00FB01E20FF31F80832F5FC6
:10E150003F4F2417350730F302C040E050E0CA01BA
:10E160000895AC0180919B0085FFFCCF70939C00CB
:10E1700080919B0085FFFCCF60939C0020E030E005
:10E180000CC080919B0085FFFCCFFA01E20FF31FCA
:10E19000808180939C002F5F3F4F2617370788F3BD
:10E1A0000895DF93CF9300D000D00F92CDB7DEB7A4
:10E1B000982F882359F081E089838FEF8A839B838E
:10E1C00063E070E0CE0101960E94B1F01EBC85B7FD
:10E1D000816085BF85B78D7F85BFE0910001F0919B
:10E1E000010109950F900F900F900F900F90CF9114
:10E1F000DF9108951092980081E080939900EBE9F7
:10E20000F0E080818D7F808388E180939A0086E0B2
:10E2100080939D000895BF92CF92DF92EF92FF927C
:10E220000F931F93CF93DF937B018C016A01E199D8
:10E23000FECF83E0F70100935B0080936800E895D0
:10E240008091680080FDFCCF40E050E060E070E02D
:10E25000BB24B394F6018081D181C0E09E01280FD8
:10E26000311D82E090E0C80ED91EDB01CA018E0D7F
:10E270009F1DA01FB11F0901FC01A0935B00B0927C
:10E280006800E89511244E5F5F4F6F4F7F4F40301D
:10E2900091E0590790E0690790E07907D9F685E0A9
:10E2A000F70100935B0080936800E8958091680017
:10E2B00080FDFCCF81E180936800E895DF91CF91EC
:10E2C0001F910F91FF90EF90DF90CF90BF90089536
:10E2D00024B714BE88E10FB6F89481BD11BC0FBEFF
:10E2E0001124D2E0C0E0F89485B7816085BF85B77E
:10E2F000826085BF8FEF90E19EBF8DBF1092980026
:10E3000091E09093990080919B008D7F80939B007A
:10E3100088E180939A0086E080939D0023FF09C0E6
:10E32000998382E98A8362E070E0CE0101960E94BF
:10E33000B1F0CE0106960E9467F08A30910511F087
:10E340000E94D1F08985813349F48A85833331F481
:10E350008B85833319F48C85873319F08FEF0E94F6
:10E36000D1F08D8590E0A0E0B0E05C019924882494
:10E370008E8590E0A0E0B0E0BA2FA92F982F8827D3
:10E38000880E991EAA1EBB1E8F85880E911CA11C8B
:10E39000B11C81E0898381E98A8366247724CC24B7
:10E3A000DD24760186E0282E312C2C0E3D1E4424DF
:10E3B0004A943AC05B826C8264E070E0CE010196C0
:10E3C0000E94B1F0C1010E9467F08C01009791F3A7
:10E3D0008E81813049F58F81813931F599858B8125
:10E3E000981711F59A858C819817F1F4F101E00FD7
:10E3F000F11FC80102C04192019621E085309207C9
:10E40000D0F3AE01455F5F4FC701B6010E940BF12B
:10E4100005501040C801A0E0B0E0C80ED91EEA1EA9
:10E42000FB1E0894611C711CC814D904EA04FB0487
:10E4300010F4572CBFCF80E98A8362E070E0CE01F0
:10E4400001960E94B1F01EBC85B7816085BF85B77B
:10E450008D7F85BFE0910001F0910101099580E079
:06E4600090E0F894FFCFEC
:040000031000E00009
:00000001FF
